:100000000C9420050C9467050C942B080C94670540
:100010000C9467050C9467050C9467050C946705B0
:100020000C9467050C9467050C941B0E0C94ED0E54
:100030000C94151D0C9467050C9467050C946705CA
:100040000C9467050C9467050C9467050C94670580
:100050000C9467050C94891D0C9467050C94670536
:100060000C9467050C9467050C9467050C94670560
:100070000C9467050C9467050C9467050C94670550
:100080000C9467050C9467050C9467050C94670540
:100090000C9467050C9467050C9467050C94670530
:1000A0000C9467050C9467050C9467055A0F7C0F38
:1000B0006A107C0F6A10C10FE40F6A1039104C10DF
:1000C0004A134A1379137913D71315142F162F16C1
:1000D0002E142F162F152F1503162F162F161A163E
:1000E000350C12132B141A8024252668742E2A2707
:1000F0002122230815171C181E1F202F3031692DAF
:1001000039041607090A0B0D0E0F33343228807C90
:1001100079781D1B0619051110363738757D647AFC
:100120002C7B7F8040413A535455565F6061578025
:100130005C5D5E6642433C675A5B58296263598046
:10014000808080803B473D518080494A4B4C4D4EDA
:10015000463E48804452453F504F8080808080809A
:10016000253032580A00253032580A004572726F25
:10017000723A20253032580A00456E640A00732511
:100180003032583A72253032582000456E61626C28
:100190006520627265616B3A20004B6579626F6120
:1001A00072642049443A20253032580A0049424DB1
:1001B000203437303420636F6E7665727465720A4E
:1001C00000726275663A2066756C6C0A00523A25B8
:1001D000303258253032580A00533A2530325820F0
:1001E000004B6579626F6172642073746172742E62
:1001F0000A0055534220636F6E66696775726564C5
:100200002E0A000D0A696E69740A005B445D005B8A
:10021000435D003803490042004D002000340037A0
:10022000003000340020006B006500790062006F30
:1002300000610072006400200063006F006E0076B1
:10024000006500720074006500720000000E037407
:10025000002E006D002E006B002E0000000403092C
:100260000409027400040100A03209040000010323
:10027000010100092111010001224000070581034D
:1002800008000A090401000103010200092111010B
:100290000001224D000705820308000A090402003C
:1002A00001030000000921110100012236000705A9
:1002B000830308000A090403000203000000092167
:1002C0001101000122220007058403200001070517
:1002D00004032000011201100100000008EDFE07D8
:1002E000470100010200010631FF0974A1010975EF
:1002F000150026FF00952075088102097615002655
:10030000FF00952075089102C005010980A10185B3
:100310000216810026B7001A81002AB700751095D1
:10032000018100C0050C0901A10185031601002609
:100330009C021A01002A9C02751095018100C005DB
:10034000010902A1010901A10005091901290515E9
:10035000002501950575018102950175038101054F
:1003600001093009311581257F950275088106093B
:10037000381581257F950175088106050C0A38021C
:100380001581257F950175088106C0C00501090604
:10039000A101050719E029E7150025019508750158
:1003A0008102950175088101050819012905950546
:1003B000750191029501750391010507190029FF47
:1003C000150026FF00950675088100C0636F6E73E7
:1003D000756D65723A20253034580A00737973744C
:1003E000656D3A20253034580A000A00253032580D
:1003F00020006B6579626F6172643A20004C45445D
:100400003A20253032580A00253032583A2025301B
:10041000386225730A00722F63203031323334354D
:1004200036370A00290A002575002F002575005D62
:100430002800256400200025640020002564002099
:10044000002564007C0025303258006D6F7573659F
:100450006B6579205B62746E7C78207920762068E9
:100460005D287265702F61636C293A205B006D6BAB
:100470005F776865656C5F74696D655F746F5F6DEC
:100480006178203D2025640A006D6B5F77686565A3
:100490006C5F6D61785F7370656564203D202564D5
:1004A0000A006D6B5F74696D655F746F5F6D617875
:1004B000203D2025640A006D6B5F6D61785F73706D
:1004C000656564203D2025640A006D6B5F696E746C
:1004D000657276616C203D2025640A006D6B5F6457
:1004E000656C6179203D2025640A006D6B5F77683B
:1004F00065656C5F74696D655F746F5F6D617820B1
:100500003D2025640A006D6B5F776865656C5F6DE3
:1005100061785F7370656564203D2025640A006D15
:100520006B5F74696D655F746F5F6D6178203D20EE
:1005300025640A006D6B5F6D61785F73706565643B
:10054000203D2025640A006D6B5F696E74657276CC
:10055000616C203D2025640A006D6B5F64656C61F1
:1005600079203D2025640A000A00257500363A20CE
:10057000776865656C5F74696D655F746F5F6D61E9
:10058000783A20000A00257500353A2077686565BD
:100590006C5F6D61785F73706565643A20000A0076
:1005A000257500343A2074696D655F746F5F6D6105
:1005B000783A20000A00257500333A206D61785F93
:1005C00073706565643A20000A00257500323A2090
:1005D000696E74657276616C286D73293A20000A21
:1005E00000257500313A2064656C6179282A313024
:1005F0006D73293A20000A092D2056616C756573C8
:10060000202D0A004D3E004D25643E20003F007322
:1006100065742064656661756C740A00433E200051
:1006200077686572652064656C74613A20637572E1
:10063000736F723D25642C20776865656C3D256479
:100640000A53656520687474703A2F2F656E2E7793
:10065000696B6970656469612E6F72672F77696B6A
:10066000692F4D6F7573655F6B6579730A000A09B1
:100670002D204D6F7573656B6579202D0A455343A9
:100680002F713A09717569740A313A0964656C61B0
:1006900079282A31306D73290A323A09696E7465F6
:1006A0007276616C286D73290A333A096D61785F3F
:1006B00073706565640A343A0974696D655F746FB7
:1006C0005F6D61780A353A09776865656C5F6D61C1
:1006D000785F73706565640A363A09776865656C9A
:1006E0005F74696D655F746F5F6D61780A0A703A57
:1006F000097072696E742076616C7565730A643A6C
:10070000097365742064656661756C74730A75702D
:100710003A092B310A646F776E3A092D310A7067F6
:1007200075703A092B31300A7067646F776E3A0939
:100730002D31300A0A7370656564203D2064656C54
:100740007461202A206D61785F7370656564202A6A
:100750002028726570656174202F2074696D655F53
:10076000746F5F6D6178290A003F004D3E200043A1
:100770003E20004C25640A000A092D20436F6E7349
:100780006F6C65202D0A4553432F713A09717569C5
:10079000740A6D3A096D6F7573656B65790A000AA5
:1007A000092D204D61676963202D0A643A0964654B
:1007B0006275670A783A096465627567206D6174CD
:1007C0007269780A6B3A096465627567206B6579AE
:1007D000626F6172640A6D3A096465627567206DC3
:1007E0006F7573650A763A0976657273696F6E0A7A
:1007F000733A097374617475730A633A09636F6EAF
:10080000736F6C65206D6F64650A302D343A096C26
:1008100061796572302D34284631302D4634290AED
:10082000506175733A09626F6F746C6F61646572C1
:100830000A003F0074696D65725F726561643332EE
:1008400028293A202530346C580A006B6579626F8C
:100850006172645F69646C653A2025580A006B65B3
:1008600079626F6172645F70726F746F636F6C3AFC
:100870002025580A00686F73745F6B6579626F6139
:1008800072645F6C65647328293A2025580A000A4F
:10089000092D20537461747573202D0A004743435A
:1008A0003A20342E392E32204156522D4C494243A3
:1008B0003A20312E382E3073766E204156525F41E9
:1008C0005243483A20617672350A004F5054494FDE
:1008D0004E533A204C554641204D4F5553454B45BC
:1008E000592045585452414B455920434F4E534F80
:1008F0004C4520434F4D4D414E44204B45594D41B1
:10090000505F53454354494F4E20343039360A0026
:100910004255494C443A20383238346433302D64DF
:1009200069727479202831363A33373A31392041A7
:1009300070722032372032303138290A005649444B
:100940003A2030784645454428742E6D2E6B2E296A
:10095000205049443A203078343730372849424DC6
:100960002034373034206B6579626F6172642063A4
:100970006F6E76657274657229205645523A203042
:1009800078303030310A00444553433A20636F6E6B
:10099000766572742049424D2034373034206B65BF
:1009A00079626F61726420746F205553420A000AA5
:1009B000092D2056657273696F6E202D0A000A6D2D
:1009C0006F7573653A206F66660A000A6D6F7573FE
:1009D000653A206F6E0A000A6B6579626F61726416
:1009E0003A206F66660A000A6B6579626F6172640D
:1009F0003A206F6E0A000A6D61747269783A206F4E
:100A000066660A000A6D61747269783A206F6E0A30
:100A1000000A64656275673A206F6E0A000A6465B1
:100A20006275673A206F66660A000A0A626F6F7421
:100A30006C6F616465722E2E2E2000433E200000F4
:100A400011241FBECFEFDAE0DEBFCDBF04B603FE38
:100A500027C08091780290917902A0917A02B0919A
:100A60007B028730904BA740B04BD1F410927802B4
:100A70001092790210927A0210927B0214BE84B70F
:100A8000877F84BF0FB6F894A89580916000886135
:100A900080936000109260000FBEE0E0F8E30995DB
:100AA00011E0A0E0B1E0E0EFFBE402C005900D92A0
:100AB000A233B107D9F722E0A2E3B1E001C01D9251
:100AC000A837B207E1F70E943E0B0C94F6250C9470
:100AD0000000FF93EF93E0913201F09133013097E2
:100AE00009F00995EF91FF910895FC0185918030FF
:100AF00011F0EFDFFBCF0895FF27E0E230E247FF80
:100B00000CC0419597FF09C0EDE260957095809506
:100B10009095611D711D811D911D27FF02C02195BA
:100B200030E350E2AA27660F771F881F991FAA1F7C
:100B3000A41710F0A41B63955A95A9F7AA3008F0E2
:100B4000A95FA05DAF93F3956115710581059105CE
:100B500041F7ED3211F4EF93F395F21718F43F9348
:100B6000F395FBCF8F91B5DFFA95E1F70895E99101
:100B7000F9918591803021F0853219F0AADFF9CF03
:100B8000089520E0E89455915532C1F3503311F4A3
:100B9000689455915A3348F4505390F3220F022E23
:100BA000220F220F200D250FF4CF0EF421958991ED
:100BB0009991533619F3533729F1533559F1BC0143
:100BC00088279927E8945C3621F489919991689453
:100BD0005591543639F446EF7EF077FF0DC08FEF14
:100BE0009FEF0AC055374AE039F0583540E121F00F
:100BF000523642E009F00895FF93EF937DDFEF91C5
:100C0000FF91B7CFFF93EF93FC0181918030B9F34F
:100C100060DFFBCFFF93EF9368DFF1CFDF93CF93DC
:100C2000CDB7DEB72596A3DFCF91DF9108950C9461
:100C30004A07E82FF0E0EC5CFE4F80810895E4E382
:100C4000F1E080E18E0F11928E13FDCF0895FF9297
:100C50000F931F93CF93DF9380915A02816080930B
:100C60005A028DEA91E00E9475050E941F062FEF3F
:100C700087EA91E6215080409040E1F700C00000F3
:100C80000E941F081F928F938AE991E09F938F9390
:100C90000E940E068BE891E00E9475050F900F9060
:100CA0000F900F908CEF0E945907882339F08FE343
:100CB0009CE90197F1F700C00000F4CFC0E0D0E05C
:100CC0000EE711E08C2F8068F82E8F2D0E945907B7
:100CD000882339F08FE39CE90197F1F700C0000009
:100CE000F4CF8FE19EE40197F1F700C000000E946D
:100CF0001F081F928F93DF93CF931F930F930E9430
:100D00000E0621960F900F900F900F900F900F905E
:100D1000CF37D105B9F68FEF0E945907882339F0F4
:100D20008FE39CE90197F1F700C00000F4CF89E759
:100D300091E0DF91CF911F910F91FF900C94750579
:100D4000CF93DF930E941F088F3F09F457C0982F5D
:100D50009F779C3778F01F928F938CE691E09F935A
:100D60008F930E940E060E941F060F900F900F9007
:100D70000F9044C090915A02C82FC695C695C6954B
:100D8000D82FD77087FF1CC090FF0CC01F928F9385
:100D900086E691E09F938F930E940E060F900F902E
:100DA0000F900F90EC2FEF70F0E0EC5CFE4F81E0C5
:100DB00090E001C0880FDA95EAF79081892B1BC07B
:100DC00090FF0CC01F928F9380E691E09F938F93CA
:100DD0000E940E060F900F900F900F90EC2FF0E0F6
:100DE000EC5CFE4F81E090E001C0880FDA95EAF7F5
:100DF000809590818923808381E001C080E0DF912C
:100E0000CF91089508959FB7F8942091480180915B
:100E10004901821761F030E0F901E65BFE4F808105
:100E20002F5F3F4F2F7133272093480101C080E08F
:100E30009FBF08955198599A08955898509A0895C7
:100E40005098589A08955198599A85E08A95F1F7E3
:100E5000000089B18695817008955098589A85E070
:100E60008A95F1F7000089B181700895CF93DF93DF
:100E7000C4E6D0E00E942307811108C0209731F01A
:100E800085E08A95F1F700002197F4CFCE01DF913C
:100E9000CF9108950E941A070E941D07E9E6F0E02D
:100EA00080818C608083E19AE99A0E941A070C94F1
:100EB0002007BF92CF92DF92EF92FF920F931F9382
:100EC000CF93DF93C82E10924701E9980E941A072A
:100ED0000E9420075998519A0CE211E00E942D07B8
:100EE00081110AC00115110549F085E08A95F1F7D5
:100EF000000001501109F2CF012B11F480E373C0FF
:100F000000E010E0D1E0D12CBB24B394C02F0E94AC
:100F10003607892B11F4C05C24C0C601002E02C024
:100F2000959587950A94E2F780FF04C0DB250E941F
:100F3000200702C00E941D0784E6E82EF12C0E94C3
:100F40002307882359F0E114F10451F085E08A95D4
:100F5000F1F7000081E0E81AF108F1CFEF2821F461
:100F6000C85BC09347014AC00F5F1F4F083011058F
:100F700069F60E943607892B11F484E334C0DD231F
:100F800029F00E94200704E610E00CC00E941D0713
:100F9000FACF0115110561F085E08A95F1F700009F
:100FA000015011090E9423078111F3CF012B11F485
:100FB00085E319C00E943607892BF9F20E942007A9
:100FC00004E610E00E942D07882351F00115110559
:100FD00049F085E08A95F1F7000001501109F2CF40
:100FE000012B21F486E38093470108C00E941A0771
:100FF0000E942007E19AE99A80E017C00E941A0730
:101000000E94200780914701813360F01F928F93E7
:1010100089ED91E09F938F930E940E060F900F90A1
:101020000F900F90E19AE99A8FEFDF91CF911F9186
:101030000F91FF90EF90DF90CF90BF9008952FB762
:10104000F89490914901809148012FBF98130C9416
:1010500003078FEF08951F920F920FB60F9211247E
:101060002F933F934F935F936F937F938F939F93B0
:10107000AF93BF93CF93DF93EF93FF93109247010A
:10108000809146018830F1F030F0893009F05CC081
:10109000C4E6D0E02EC0809145018695809345013D
:1010A0000E942D07882309F449C08091450180687A
:1010B0008093450181E090914401911180E08093FB
:1010C00044013CC00E942D07882339F081E09091B3
:1010D0004401911180E08093440180914401882370
:1010E00099F12CC0209781F185E08A95F1F70000F5
:1010F00021970E942D078111F5CFCD2B29F1409129
:101100004501CFB7F8948091490190E09C012F5F91
:101110003F4F2F71332750914801521739F0FC018E
:10112000E65BFE4F40832093490104C081EC91E0CF
:101130000E947505CFBF109247012AC080914601D9
:101140008F5F809346012AC08091460180934701BA
:101150008EEF0E945907882339F08FE99FE00197AD
:10116000F1F700C00000F4CF809145011F928F93EA
:10117000809146011F928F938DEC91E09F938F9306
:101180000E940E060F900F900F900F900F900F90EF
:10119000109246011092450110924401FF91EF9187
:1011A000DF91CF91BF91AF919F918F917F916F917F
:1011B0005F914F913F912F910F900FBE0F901F9015
:1011C00018958091760108959FB7F89410926D015B
:1011D0009FBF90916F02943009F057C09091E90041
:1011E0009F703091EC00232F217030FD20E8922B6E
:1011F00024E02093E9002091EB0020FF43C02091E0
:10120000EE0027FF3FC020916A01222321F02091A8
:10121000E80025FF37C010926A0126E03091E8000F
:1012200035FD15C030916F02343061F53091EB001F
:1012300035FD28C0215021F481E080936A0122C04D
:10124000EFE9FFE03197F1F700C00000E7CF8093AE
:10125000F1008091E80085FD0AC08091E80080FFE0
:10126000FCCF8091E8008E778093E80006C08FB7AE
:10127000F89421E020936D018FBF9F709093E90057
:1012800080E008959F709093E9008FEF0895CF93C9
:10129000DF9300D01F92CDB7DEB79C0180916F0223
:1012A000843019F593E099833B832A839093E90076
:1012B0008FEF9091E800815095FD06C095ED9A95CD
:1012C000F1F700008111F5CF8091E80085FF0DC096
:1012D00040E050E063E070E0CE0101960E940B0C0C
:1012E0008091E8008E778093E8000F900F900F9028
:1012F000DF91CF910895CF93DF9300D01F92CDB7A8
:10130000DEB720916F02243021F522E029839B83F0
:101310008A8383E08093E9008FEF9091E800815009
:1013200095FD06C095ED9A95F1F700008111F5CF76
:101330008091E80085FF0DC040E050E063E070E080
:10134000CE0101960E940B0C8091E8008E7780936D
:10135000E8000F900F900F90DF91CF9108952091AA
:101360006F022430F1F422E02093E9002FEF309156
:10137000E800215035FD06C035ED3A95F1F7000043
:101380002111F5CF2091E80025FF0BC040E050E08F
:1013900065E070E00E940B0C8091E8008E778093EE
:1013A000E8000895CF93DF9320916F02243039F540
:1013B00021E02093E9002FEF3091E800215035FD26
:1013C00006C035ED3A95F1F700002111F5CF2091D7
:1013D000E80025FF14C0EC0140E050E068E070E058
:1013E0000E940B0C8091E8008E778093E80088E0E3
:1013F000FE01AEE6B1E001900D928A95E1F7DF9132
:10140000CF9108958FE092E00E94750580916E0261
:10141000811109C00E94A00D0E94FD0D8091E20083
:1014200084608093E20008958BE092E00E9475054D
:1014300010926E020895089520916B012F5F822F04
:1014400062E30E94BC25992319F020936B01089553
:1014500010926B0180916D01882371F180916F0270
:10146000843041F58091E9008F702091EC00922F3B
:10147000917020FD90E8892B94E09093E900909181
:10148000EB0090FF14C09091EE0097FF10C0909178
:10149000E80095FF03C01092F100F9CF9091E800A9
:1014A00090FF05C09091E8009E779093E8008F70C0
:1014B0008093E90010926D01089542E061EC81E0B3
:1014C0000E941A0D42E061EC82E00E941A0D42E097
:1014D00061EC83E00E941A0D42E261EC84E00C941E
:1014E0001A0D80917102833009F453C030F48130B9
:1014F00071F0823009F48CC008958A3009F478C004
:101500008B3009F45EC0893009F09AC020C0809108
:101510007002813A09F094C08091E800877F80933F
:10152000E8008091740290917502892B21F468E0A3
:101530008EE691E003C060E080E090E070E00E9401
:10154000560C8091E8008B778093E8000895809195
:101550007002813209F074C080917402909175021A
:10156000892B09F06DC08091E800877F8093E800A7
:101570008091E80082FD05C080916F028111F8CF53
:101580005FC08091F100809376018091E8008B77B5
:1015900053C080917002813A09F052C08091740268
:1015A00090917502892B09F04BC08091E800877FEC
:1015B0008093E8008091E80080FFFCCF80910A01D1
:1015C00036C0809170028132D9F580917402909179
:1015D0007502892BA9F58091E800877F8093E80048
:1015E0000E944F0D8091720280930A010C94511653
:1015F00080917002813221F58091E800877F80938D
:10160000E8000E944F0D8091730280937701089546
:1016100080917002813AA1F48091E800877F8093E5
:10162000E8008091E80080FFFCCF809177018093F3
:10163000F1008091E8008E778093E8000C944F0DC4
:101640000895089508958091760180936C01109219
:10165000760180E00E9402070E941F060C9451163A
:101660000C94230B0E94D41C80916D02882329F0D6
:101670000E94FD1C81110C94F50B089584B7877F9F
:1016800084BF0FB6F894A89580916000886180931C
:101690006000109260000FBE90E080E80FB6F894F2
:1016A00080936100909361000FBE84EE98E00E94E9
:1016B000A51C83E092E00E9475050E94210B0E9408
:1016C00043110E94A00D0E94FD0D8091E2008460F4
:1016D0008093E200789480916F028430E1F781ED8D
:1016E00097E0019739F0EFE9FFE03197F1F700C09B
:1016F0000000F7CF82EF91E00E9475050E9445112E
:1017000080E091E00E94821081EE91E00E947505D8
:101710000E94220B80916F02853019F40E94320BD7
:10172000F9CF0E944911F6CF0E94111D80916C01E2
:101730008093760108950C94940B292F332723303E
:101740003105C9F064F42130310581F022303105D2
:1017500009F043C084E790E021E632E042C0213244
:101760003105F1F02232310541F137C082E190E0DC
:1017700025ED32E036C099278130910541F0823065
:10178000910541F0892B49F5EDE5F2E005C0EDE466
:10179000F2E002C0E3E1F2E0849190E09F0121C019
:1017A0006430D8F4E62FF0E0EE0FFF1FE15EFE4F4D
:1017B0002081318189E090E014C0643070F470E0E1
:1017C000FB01EE0FFF1FE95EFE4F20813181FB011F
:1017D000ED5EFE4F808190E004C080E090E020E06C
:1017E00030E0FA0131832083089580E189BD82E1F0
:1017F00089BD09B400FEFDCF8091D8008F7D809314
:10180000D8008091E00082608093E0008091E00049
:1018100081FDFCCF0895CF92DF92EF92FF920F935C
:101820001F93CF93DF93EC018B016A010E946E0D31
:10183000811133C0C114D10439F0F6018081918146
:10184000081B190BC80FD91FE12CF12C011511052C
:1018500019F18091E80085FD16C08091E8008E772F
:101860008093E800C114D10449F0F6018081918190
:10187000E80EF91EF182E08285E00FC00E946E0D35
:10188000882321F30AC089918093F1000150110946
:10189000FFEFEF1AFF0ADACF80E0DF91CF911F91BF
:1018A0000F91FF90EF90DF90CF90089520917602F6
:1018B000309177022617370748F06115710539F422
:1018C0002091E8002E772093E80001C0B90140E0A4
:1018D00061157105A9F120916F02222309F443C01B
:1018E000253009F442C02091E80023FD40C020913A
:1018F000E80022FD32C02091E80020FFE9CF4091AE
:10190000F3002091F20030E0342BFC01CF0161158F
:10191000710559F02830310540F481918093F10030
:10192000615071092F5F3F4FF1CF41E02830310501
:1019300009F040E02091E8002E772093E800C8CF1E
:101940004111C9CF0AC080916F02882361F08530B0
:1019500061F08091E80083FD0AC08091E80082FF79
:10196000F2CF80E0089582E0089583E0089581E059
:10197000089520917602309177022617370748F0B4
:101980006115710539F42091E8002E772093E80065
:1019900001C0B901FC0120E06115710591F1809150
:1019A0006F02882309F440C0853009F43FC080915C
:1019B000E80083FD3DC08091E80082FD2FC080914A
:1019C000E80080FFE9CF2091F3008091F20090E0E1
:1019D000922B6115710559F08830910540F42491DE
:1019E0002093F1003196615071090196F2CF21E008
:1019F000089709F020E08091E8008E778093E80056
:101A0000CBCF2111CCCF0AC080916F02882361F027
:101A1000853061F08091E80083FD0AC08091E80084
:101A200082FFF2CF80E0089582E0089583E0089578
:101A300081E00895982F973058F59093E900981712
:101A400039F07091EC002091ED005091F00003C04E
:101A5000242F762F50E021FF19C03091EB003E7FFC
:101A60003093EB003091ED003D7F3093ED003091ED
:101A7000EB0031603093EB007093EC002093ED00AD
:101A80005093F0002091EE0027FF07C09F5FD3CF57
:101A90008F708093E90081E0089580E0089580913F
:101AA000700287FF11C08091E80082FD05C080911F
:101AB0006F028111F8CF11C08091E8008B770BC0C5
:101AC00080916F02882349F08091E80080FFF8CF71
:101AD0008091E8008E778093E80008952091E400DB
:101AE0003091E50095E64091EC00842F817040FF35
:101AF00022C08091E80080FD1CC080916F02882385
:101B000091F0853091F08091EB0085FD10C04091FF
:101B1000E4005091E5004217530729F39A019150D0
:101B200011F784E0089582E0089583E0089581E04C
:101B3000089580E008954091E80042FFDECF0895C7
:101B40000E940E0E0E94160EE0EEF0E08081816091
:101B50008083E8EDF0E080818F77808319BCA7ED6A
:101B6000B0E08C918E7F8C9380818F7E80831092E9
:101B70006E0208950F931F93CF93DF930E940E0E72
:101B80000E94160EC8EDD0E088818F778883888107
:101B90008068888388818F7D888319BC10926F024A
:101BA00010926B0210926D0210926C0200EE10E027
:101BB000F80180818B7F808388818160888342E007
:101BC00060E080E00E941A0DE1EEF0E080818E7FFF
:101BD0008083E2EEF0E08081816080838081886094
:101BE0008083F80180818E7F8083888180618883F3
:101BF000DF91CF911F910F910895E8EDF0E0808182
:101C00008F7E8083E7EDF0E080818160808384E0D7
:101C100082BF81E080936E020C94BA0DE8EDF0E093
:101C200080818E7F80831092E20008951092DA0006
:101C30001092E10008951F920F920FB60F92112497
:101C40002F933F934F935F936F937F938F939F93C4
:101C5000AF93BF93EF93FF938091E10082FF0BC09E
:101C60008091E20082FF07C08091E1008B7F80932A
:101C7000E1000E941C0A8091DA0080FF1FC0809161
:101C8000D80080FF1BC08091DA008E7F8093DA003D
:101C90008091D90080FF0DC080E189BD82E189BDBE
:101CA00009B400FEFDCF81E080936F020E94020A1A
:101CB00005C019BC10926F020E94140A8091E100C5
:101CC00080FF19C08091E20080FF15C08091E20082
:101CD0008E7F8093E2008091E20080618093E20039
:101CE0008091D80080628093D80019BC85E08093F1
:101CF0006F020E94300B8091E10084FF30C0809120
:101D0000E20084FF2CC080E189BD82E189BD09B475
:101D100000FEFDCF8091D8008F7D8093D800809108
:101D2000E1008F7E8093E1008091E2008F7E8093BE
:101D3000E2008091E20081608093E20080916B027A
:101D4000882311F084E007C08091E30087FD02C082
:101D500081E001C083E080936F020E949B0B809121
:101D6000E10083FF29C08091E20083FF25C08091BC
:101D7000E100877F8093E10082E080936F02109200
:101D80006B028091E1008E7F8093E1008091E20000
:101D90008E7F8093E2008091E20080618093E20078
:101DA00042E060E080E00E941A0D8091F0008860BF
:101DB0008093F0000E941B0AFF91EF91BF91AF91B9
:101DC0009F918F917F916F915F914F913F912F9153
:101DD0000F900FBE0F901F9018951F920F920FB685
:101DE0000F9211242F933F934F935F936F937F93A1
:101DF0008F939F93AF93BF93CF93DF93EF93FF9313
:101E0000C091E900CF708091EC00D82FD17080FD97
:101E1000D0E81092E9008091F000877F8093F00075
:101E200078940E94310F1092E9008091F000886050
:101E30008093F000CD2BCF70C093E900FF91EF911C
:101E4000DF91CF91BF91AF919F918F917F916F91D2
:101E50005F914F913F912F910F900FBE0F901F9068
:101E600018951F93CF93DF93CDB7DEB7AA970FB620
:101E7000F894DEBF0FBECDBFE0E7F2E088E08E0F42
:101E80009091F10091938E13FBCF0E94710A809183
:101E9000E80083FF1FC18091700290917102492F69
:101EA00050E04A30510508F015C1FA01EA5AFF4FD7
:101EB0000C94DC25803881F0823809F00BC18091C8
:101EC00074028F708093E9008091EB0085FB882776
:101ED00080F91092E90006C080916C0290916D0229
:101EE000911182609091E800977F9093E800809331
:101EF000F1001092F100C8C0282F2D7F09F0EAC030
:101F0000882319F0823061F0E5C08091720281303F
:101F100009F0E0C0933009F080E080936D022BC09F
:101F200080917202811127C0809174028F7009F430
:101F3000D1C08093E9002091EB0020FF1CC09330BA
:101F400021F48091EB00806214C09091EB009061CD
:101F50009093EB0021E030E0A90102C0440F551F2F
:101F60008A95E2F74093EA001092EA008091EB0034
:101F700088608093EB001092E9008091E800877FF1
:101F800086C08111A7C0109172021F778091E30073
:101F90008078812B8093E3008091E800877F809395
:101FA000E8000E944F0D8091E80080FFFCCF8091F7
:101FB000E30080688093E300111102C082E001C059
:101FC00083E080936F0286C08058823008F082C020
:101FD00080917202909173028C3D53E0950779F5E0
:101FE00083E08A838AE289834FB7F894DE011396EF
:101FF00020E03EE051E2E32FF0E050935700E491FF
:1020000020FF03C0E295EF703F5FEF708E2F90E0EE
:10201000EA3010F0C79601C0C0968D939D932F5F54
:10202000243149F74FBF8091E800877F8093E80013
:102030006AE270E0CE0101960E94560C14C0AE0117
:102040004F5F5F4F609174020E949D0BBC01892B12
:1020500009F440C09091E800977F9093E80089814F
:102060009A810E94B90C8091E8008B778093E800F8
:1020700031C0803879F58091E800877F8093E8004F
:1020800080916B028093F1008091E8008E778093BD
:10209000E8000E944F0D1EC081111CC09091720279
:1020A0009230C0F48091E800877F8093E80090939D
:1020B0006B020E944F0D80916B02811106C08091CE
:1020C000E30087FD02C081E001C084E080936F02DD
:1020D0000E945D0A8091E80083FF0AC08091E800B9
:1020E000877F8093E8008091EB0080628093EB0013
:1020F000AA960FB6F894DEBF0FBECDBFDF91CF9189
:102100001F91089590937D0180937C010895E09143
:102110007C01F0917D01309721F00190F081E02D5C
:10212000099480E00895EF92FF920F931F93CF934D
:10213000DF93E0917C01F0917D013097B1F18C014A
:102140000280F381E02D099580915A0282FF2DC013
:1021500080FF04C082EF93E00E947505E80118E05B
:102160008CEEE82E83E0F82E80915A0280FF0BC09F
:1021700088811F928F93FF92EF920E940E060F901C
:102180000F900F900F90115021961111EDCF80916B
:102190005A0280FF0AC08AEE93E0DF91CF911F912F
:1021A0000F91FF90EF900C947505DF91CF911F91E7
:1021B0000F91FF90EF900895E0917C01F0917D01E7
:1021C000309721F00480F581E02D09940895CF9394
:1021D000DF93EC0180917A0190917B01C817D907B8
:1021E00009F1D0937B01C0937A01E0917C01F091D9
:1021F0007D013097B9F00680F781E02DCE01099579
:1022000080915A0282FF0EC080FF0CC0DF93CF93F3
:102210008CED93E09F938F930E940E060F900F908A
:102220000F900F90DF91CF910895CF93DF93EC0142
:102230008091780190917901C817D90709F1D0935D
:102240007901C0937801E0917C01F0917D01309794
:10225000B9F00084F185E02DCE01099580915A02F4
:1022600082FF0EC080FF0CC0DF93CF938CEC93E015
:102270009F938F930E940E060F900F900F900F90D8
:10228000DF91CF9108950C9417060E943E1D0C9487
:102290002706BF92CF92DF92EF92FF920F931F9388
:1022A000CF93DF9300D000D01F92CDB7DEB70E944E
:1022B000A0060FE711E0F12C8F2D0E941906B82E11
:1022C000F801C080C82639F4F3940F5F1F4FF0E186
:1022D000FF12F2CF30C080915A0281FD0E94EE11B0
:1022E000D12CEE24E3948E2D8C21F9F0D982FA8240
:1022F00081E09E2D9B2109F480E08B830E94471D85
:102300008160782F9D838C8349815A816B818D8177
:102310000E94241249815A816B817C818D810E94A7
:10232000C11CF80190819E259083D394EE0CF8E0B7
:10233000DF12D9CFC9CF8FEF89838A831B820E9496
:10234000471D8160782F9D838C8349815A816B81E1
:102350008D810E9424120E94C01C0E9408201091AE
:102360007E010E948710181741F10E948710809308
:102370007E0190915A0292FF0EC090FF0CC01F92F6
:102380008F938DEF93E09F938F930E940E060F9093
:102390000F900F900F9080917E010F900F900F90F3
:1023A0000F900F90DF91CF911F910F91FF90EF90C1
:1023B000DF90CF90BF900C94D21C0F900F900F9095
:1023C0000F900F90DF91CF911F910F91FF90EF90A1
:1023D000DF90CF90BF9008950C940207EF92FF9288
:1023E0000F931F93CF93DF9386E194E00E947505CE
:1023F000C0E0D0E087E2E82E81E0F82E08E014E0AB
:102400008C2F0E9419060E94AA1CFF92EF921F9225
:102410008F93DF93CF931F930F930E940E06219605
:102420008DB79EB708960FB6F8949EBF0FBE8DBFAE
:10243000C031D10529F7DF91CF911F910F91FF9006
:10244000EF90089508950895CF93DF93CDB7DEB749
:102450002B970FB6F894DEBF0FBECDBF942F4F83DE
:10246000252F588769877A878B874A855B85452B17
:1024700021F02F3F09F59F3FF9F4DE01119686E028
:10248000FD0111928A95E9F785E0FE0137960190EA
:102490000D928A95E1F749815A816B817C818D810A
:1024A0009E810E942E192B960FB6F894DEBF0FBEA8
:1024B000CDBFDF91CF9108954F81588569857A8589
:1024C0008B850E94C11CD9CFCF93882309F465C0A6
:1024D000C82F8CEF8C0F813A20F080E58C0F8E3264
:1024E00048F48C2F0E943223811157C08C2F0E94F8
:1024F000061C0CC080E28C0F883058F4C77081E055
:1025000001C0880FCA95EAF70E94451CCF910C9430
:102510007F1C8BE58C0F833078F4C53A29F0C63ADE
:1025200031F083E890E005C081E890E002C082E8E5
:1025300090E0CF910C94E71088E58C0F853168F519
:10254000C83A89F0C93A91F0CA3A99F0CB3AA1F069
:10255000CC3AA9F0CD3AB1F0CE3AB9F0CF3AC1F0C9
:1025600080E090E017C082EE90E014C089EE90E029
:1025700011C08AEE90E00EC085EB90E00BC086EBB8
:1025800090E008C083EB90E005C084EB90E002C0CF
:1025900087EB90E0CF910C941511CF91089588238B
:1025A00049F19CEF980F913A20F090E5980F9E32F8
:1025B00018F40E94231C0DC090E2980F983058F434
:1025C000877091E001C0990F8A95EAF7892F0E94E0
:1025D0004B1C0C947F1C9BE5980F933020F480E0FB
:1025E00090E00C94E710885A853120F480E090E068
:1025F0000C9415110895882321F00E94451C0C9419
:102600007F1C0895882321F00E944B1C0C947F1C92
:102610000895BF92CF92DF92EF92FF920F931F9394
:10262000CF93DF9300D000D000D0CDB7DEB725E048
:10263000FC01DE01119601900D922A95E1F7FC0153
:1026400040815181028163817481258122952F709F
:102650006115710509F403C35F3F19F44F3F09F495
:10266000FEC26C01862F7D836C83602F782F8D8155
:102670002E830E948A1B182FB92E0E94891B0E944C
:10268000791AEB2DE295EF70F0E0E05AFF4F2E81C2
:102690000C94DC258B2D807F9B2D9F70F92E882339
:1026A00019F0F29490EFF922002349F0FF2009F489
:1026B00083C28F2D0E94581C0E947F1C7DC2812FD7
:1026C0000E94CF12FF2009F4CAC28F2D0E945E1C07
:1026D00026960FB6F894DEBF0FBECDBFDF91CF9127
:1026E0001F910F91FF90EF90DF90CF90BF900C94CF
:1026F0007F1C8B2D807F9B2D9F70F92E803219F0CF
:10270000F29480EFF822112319F0113009F12AC058
:102710000023B1F08F2D222351F1213041F526966F
:102720000FB6F894DEBF0FBECDBFDF91CF911F91E2
:102730000F91FF90EF90DF90CF90BF900C94681CAA
:10274000222319F0213009F48AC20E946B1C2DC08B
:102750000023F1F0263008F082C20E94421C8F2133
:1027600029F023C00023F9F0211116C08F2D2696E1
:102770000FB6F894DEBF0FBECDBFDF91CF911F9192
:102780000F91FF90EF90DF90CF90BF900C94FB12D1
:10279000253008F064C209C0F601858180FF0CC2B3
:1027A0008F708583E3CF21111CC28F2D83C12B2D08
:1027B00026952695237030E02115310521F0213032
:1027C0003105D1F04CC2002321F0812F9B2D937055
:1027D00002C080E090E026960FB6F894DEBF0FBEF0
:1027E000CDBFDF91CF911F910F91FF90EF90DF90C0
:1027F000CF90BF900C94E710002321F0812F9B2DE8
:10280000937002C080E090E026960FB6F894DEBF89
:102810000FBECDBFDF91CF911F910F91FF90EF9031
:10282000DF90CF90BF900C941511812F002319F0E9
:102830000E948E1E02C00E94F61E26960FB6F894C5
:10284000DEBF0FBECDBFDF91CF911F910F91FF90E3
:10285000EF90DF90CF90BF900C947B1F8B2D8370F7
:1028600009F07BC00111FBC1812F8295869587708D
:10287000880F880F912F9F70C92ED12CE12CF12C3D
:10288000082E04C0CC0CDD1CEE1CFF1C0A94D2F7F1
:1028900014FF12C04FE050E060E070E004C0440F4D
:1028A000551F661F771F8A95D2F7CB01BA01609535
:1028B00070958095909503C060E070E0CB012B2D62
:1028C000269526952370422F50E042305105D9F0CD
:1028D0004330510569F16C297D298E299F294130AA
:1028E000510551F126960FB6F894DEBF0FBECDBF4D
:1028F000DF91CF911F910F91FF90EF90DF90CF90DC
:10290000BF900C949E1A6C297D298E299F292696AA
:102910000FB6F894DEBF0FBECDBFDF91CF911F91F0
:102920000F91FF90EF90DF90CF90BF900C94B81A6A
:102930000E949E1AC701B60126960FB6F894DEBF14
:102940000FBECDBFDF91CF911F910F91FF90EF9000
:10295000DF90CF90BF900C94841A002319F08B2D38
:10296000817001C08695882309F479C1812F8295F1
:1029700086958770880F880F912F9F70C92ED12C54
:10298000E12CF12C082E04C0CC0CDD1CEE1CFF1C2D
:102990000A94D2F714FF12C04FE050E060E070E0FC
:1029A00004C0440F551F661F771F8A95D2F7CB01CD
:1029B000BA01609570958095909503C060E070E0D5
:1029C000CB012B2D269526952370422F50E04230C7
:1029D0005105D9F04330510569F16C297D298E29C3
:1029E0009F294130510551F126960FB6F894DEBF6C
:1029F0000FBECDBFDF91CF911F910F91FF90EF9050
:102A0000DF90CF90BF900C94651B6C297D298E2997
:102A10009F2926960FB6F894DEBF0FBECDBFDF917B
:102A2000CF911F910F91FF90EF90DF90CF90BF90CB
:102A30000C94771B0E94651BC701B60126960FB642
:102A4000F894DEBF0FBECDBFDF91CF911F910F91E4
:102A5000FF90EF90DF90CF90BF900C94531B103FEE
:102A6000D1F128F480E4810F803250F0A0C0123FF1
:102A700009F462C008F44BC0133F09F472C097C058
:102A8000F12FF071FF2E8B2D8F71002351F00E94DA
:102A9000EC1A812FFF2019F08295807F68CE8F700D
:102AA00066CE0E940D1B812FFF2019F08295807F3A
:102AB00001C08F7026960FB6F894DEBF0FBECDBF53
:102AC000DF91CF911F910F91FF90EF90DF90CF900A
:102AD000BF900C9402130023B1F0253008F0BFC062
:102AE0008B2D8F7126960FB6F894DEBF0FBECDBF2B
:102AF000DF91CF911F910F91FF90EF90DF90CF90DA
:102B0000BF900C94321B263008F0A9C0E9CF0023F7
:102B1000A9F08B2D8F7126960FB6F894DEBF0FBEED
:102B2000CDBFDF91CF911F910F91FF90EF90DF907C
:102B3000CF90BF900C94EC1A002359F38B2D8F711A
:102B400026960FB6F894DEBF0FBECDBFDF91CF91B2
:102B50001F910F91FF90EF90DF90CF90BF900C945A
:102B60000D1B002399F08B2D8F7126960FB6F894CC
:102B7000DEBF0FBECDBFDF91CF911F910F91FF90B0
:102B8000EF90DF90CF90BF900C94D71A26960FB697
:102B9000F894DEBF0FBECDBFDF91CF911F910F9193
:102BA000FF90EF90DF90CF90BF900C94D21A00234B
:102BB000A9F0222309F4ADCF812F26960FB6F89401
:102BC000DEBF0FBECDBFDF91CF911F910F91FF9060
:102BD000EF90DF90CF90BF900C946412222309F401
:102BE000ADCF812F26960FB6F894DEBF0FBECDBFB6
:102BF000DF91CF911F910F91FF90EF90DF90CF90D9
:102C0000BF900C94CF124B2D4F70612FC6010E94C4
:102C1000081E26960FB6F894DEBF0FBECDBFDF911B
:102C2000CF911F910F91FF90EF90DF90CF90BF90C9
:102C30000C94D2194B2D4F70612FC60126960FB6FA
:102C4000F894DEBF0FBECDBFDF91CF911F910F91E2
:102C5000FF90EF90DF90CF90BF900C940B1E2696C4
:102C60000FB6F894DEBF0FBECDBFDF91CF911F919D
:102C70000F91FF90EF90DF90CF90BF9008950E944A
:102C8000651C0E94341C0E947F1C0E94AD200E9483
:102C90007B1F80E090E00E94E71080E090E00C94C1
:102CA00015110E94551C0C943F16CF93DF9300D052
:102CB00000D01F92CDB7DEB7942F4983252F5A83BA
:102CC0006B837C838D834C815D81452B39F12F3F54
:102CD00011F49F3F19F149815A816B817C818D816B
:102CE0000E948A1B292F22952F7030E02C3031054D
:102CF00004F52A3031055CF42250310922303105C7
:102D000068F4853A80F4843090F4823080F0883E14
:102D100038F4803E60F48450813A48F080E014C07A
:102D2000803FE1F704C090E2980F983080F781E08F
:102D30000BC02C30310521F493FB882780F904C0A7
:102D40002F303105C9F3EACF0F900F900F900F90FD
:102D50000F90DF91CF910895CF93DF9300D000D0F3
:102D60001F92CDB7DEB70F900F900F900F900F907E
:102D7000DF91CF910895CF93DF9300D000D000D0A2
:102D8000CDB7DEB726960FB6F894DEBF0FBECDBF27
:102D9000DF91CF9108951F93CF93DF93C0918F015F
:102DA00016E080919001C81799F0D0E01C9FF001C7
:102DB0001D9FF00D1124EF56FE4F4081518162811D
:102DC0007381848195810E94BB162196C770E9CFDB
:102DD000DF91CF911F9108954091C1015091C2019F
:102DE0006091C3017091C4018091C5019091C601A9
:102DF0000C94BB168091C60182958F7009F054C067
:102E00008091C301882309F44FC080918F01A09164
:102E100090016091C1017091C2014091C401509133
:102E2000C501B6E08A1709F43FC090E0411551058D
:102E3000C1F17F3F11F46F3FA1F1B89FF001B99F3D
:102E4000F00D1124EF56FE4F218172132AC020810C
:102E5000621327C02281211124C0238134812417C9
:102E6000350710F421503109241B350B283C31055E
:102E7000C0F42091C6012F7020612093C60126E086
:102E8000289FF001299FF00D1124EA56FE4F808102
:102E90008F708061808381EC91E00E9409130C9413
:102EA000CB1601968770BECF0895BF92CF92DF9266
:102EB000EF92FF920F931F93CF93DF93CDB7DEB7BF
:102EC00061970FB6F894DEBF0FBECDBF7C0185E0E1
:102ED000F701DE011D9601900D928A95E1F7D70169
:102EE0004C9111965C9111971296DC901297139663
:102EF0000D911C9114973091C1016091C201809194
:102F0000C4019091C501009709F477C16F3F19F48E
:102F10003F3F09F472C1B090C301BB2009F4C5C0A2
:102F20002091C6010817190728F0F801E81BF90BD2
:102F3000CF0104C080959095800F911FCC24C3943D
:102F4000883C910580F0C12C207F09F0CCC0702F07
:102F5000198B088B6D2D89890E94AC1681EC91E04C
:102F60000E940913B6C0822F807F09F047C0651305
:102F700014C0341312C0D11010C02F7020612093E0
:102F8000C6010E94EC1681EC91E00E940913809129
:102F9000C601D70115968C932FC00115110519F1A3
:102FA0005F3F11F44F3FF9F0CD2CD1101CC0809140
:102FB0008F012091900136E0821709F45CC090E007
:102FC000389FF001399FF00D1124EF56FE4F6181BB
:102FD000561306C06081461303C06281611103C0AD
:102FE00001968770E9CFCD2CDD2009F426C18091B0
:102FF000C60181608093C601C12C1FC1651308C042
:10300000341306C0D11004C08091C601D701C9C0D5
:103010004D875E87DF86702F198B088B6D2D898910
:103020000E9455168823E9F1DD20D9F12091C601CF
:10303000822F82958F7090E0029774F08091C10189
:103040009091C20198878F8319861B870A872C87E6
:10305000CE0107960E94091386E0F701A1ECB1E0CA
:1030600001900D928A95E1F70E94FA160E94EC16E3
:10307000CC24C394E2C0702F198B088B60E089893F
:103080000E948A1B292F22952F7030E022303105B3
:103090000CF0C7C09F7009F0C1C0805E883008F492
:1030A000CCC0C7010E940913E3CF0817190708F421
:1030B00056C0F801E81BF90BCF01883C910508F4D4
:1030C00053C0C12C702F198B088B6D2D89890E94DC
:1030D000AC16E1ECF1E086E0DF011D928A95E9F79C
:1030E0000E94EC16AAC0651314C0341312C0D1108C
:1030F00010C08091C601F7018583C7010E940913A2
:1031000086E0E1ECF1E0DF011D928A95E9F7CB2C36
:1031100094C04D875E87DF86702F198B088B6D2DCD
:1031200089890E945516882309F4BBCFDD2009F454
:10313000B8CF2091C601822F82958F7090E00297C0
:103140000CF48ACF8091C1019091C2019A83898346
:103150001B821D830C832E83CE0101967BCF80952D
:103160009095800F911FA9CFCD2CDD2009F499CF28
:1031700065132EC034132CC02091C60120FD1FC042
:10318000822F82958F70D9F0D70115962C931597C1
:103190008F3049F08F5F982F9295907F822F8F709C
:1031A000892B15968C93C7010E94091386E0F701BD
:1031B000A1ECB1E001900D928A95E1F791CF86E004
:1031C000F701A1ECB1E001900D928A95E1F735C0CD
:1031D0004D875E87DF86702F198B088B6D2D89894F
:1031E0000E945516811138CF8091C601816080936D
:1031F000C601C7010E94091320C0DD2009F451CF88
:103200004D875E87DF86702F198B088B6D2D89891E
:103210000E945516882309F444CF1ECF81113DCF5B
:103220000CC0243031050CF03CCF9F7009F435CF31
:10323000F7019581907F09F030CF8C2D61960FB604
:10324000F894DEBF0FBECDBFDF91CF911F910F91DC
:10325000FF90EF90DF90CF90BF9008951F93CF9392
:10326000DF93CDB7DEB72C970FB6F894DEBF0FBE55
:10327000CDBF4F83588769877A878B879C87CE011C
:1032800007960E945517882369F08F8198852A85B3
:103290003B85232BF1F19F3F09F063C08F3F09F07D
:1032A00060C037C086E0FE013796DE0111960190BE
:1032B0000D928A95E1F76F817885EA85FB853097D5
:1032C00041F17F3F11F46F3F21F12091900130E0F7
:1032D000C90101968770992740918F0150E08417AA
:1032E000950709F447C069837A83FD83EC8396E0F0
:1032F000929FD001939FB00D1124AF56BE4FFE0197
:10330000319601900D929A95E1F7809390010E9479
:10331000CB1616E080918F01909190018917C1F131
:10332000189FC00111248F569E4F0E945517882365
:1033300079F1E0918F011E9FF0011124EF56FE4FAD
:103340004081518162817381848195810E94BB1685
:1033500080918F0190E001968770992780938F016B
:10336000D9CF4F81588569857A858B859C850E9448
:10337000BB16CFCF0E9451161092900110928F0170
:10338000E1ECF1E086E0DF011D928A95E9F7C1CF1B
:103390002C960FB6F894DEBF0FBECDBFDF91CF9154
:1033A0001F910895DF92EF92FF920F931F93CF9397
:1033B000DF93FC01892B09F48AC0E12CF12CDD2478
:1033C000D394EF0121968491853709F461C058F4B4
:1033D000843708F04EC0843008F06AC08130D1F0E4
:1033E000823071F174C0883709F45DC050F48637BB
:1033F00009F455C0873709F06AC08E2D0E94521C0F
:1034000054C09CE7980F903708F061C08F770E94F6
:10341000CF1250C08F010E5F1F4FFE01849190E2CA
:10342000980F983050F48770FD2D01C0FF0F8A95DA
:10343000EAF78F2F0E94581C14C00E94641213C018
:103440008F010E5F1F4FFE01C49180E28C0F883008
:1034500060F4C7708D2D01C0880FCA95EAF70E94ED
:103460005E1C0E947F1CE80125C08C2F0E94CF1299
:10347000FACF9F012E5F3F4FFE01C491CC2369F02C
:103480008FE99FE00197F1F700C00000C150F6CF2F
:103490009F012E5F3F4FFE01F490E9010BC00E9497
:1034A000421CE82E07C00E94551C0E947F1C02C0CF
:1034B0000E9464128F2D882341F0EFE9FFE03197DD
:1034C000F1F700C000008150F6CFFE017ACFDF9106
:1034D000CF911F910F91FF90EF90DF90089560932F
:1034E0004702709348028093490290934A020C94D9
:1034F000D11C089560934B0270934C0280934D024F
:1035000090934E020C94D01C0F931F9300914B028A
:1035100010914C0220914D0230914E02602B712B84
:10352000822B932B60934B0270934C0280934D023D
:1035300090934E021F910F910C94D01C0F931F93E8
:1035400000914B0210914C0220914D0230914E029D
:10355000602371238223932360934B0270934C0268
:1035600080934D0290934E021F910F910C94D01CAA
:103570000F931F9300914B0210914C0220914D022A
:1035800030914E02602771278227932760934B0268
:1035900070934C0280934D0290934E021F910F91B5
:1035A0000C94D01C60E070E0CB010C946F1A0F9368
:1035B0001F9341E050E060E070E08A019B0104C08D
:1035C000000F111F221F331F8A95D2F7C901B801BE
:1035D0001F910F910C946F1A0F931F9341E050E0CD
:1035E00060E070E004C0440F551F661F771F8A9586
:1035F000D2F78091470290914802A0914902B09180
:103600004A028A019B01082B192B2A2B3B2BC9014B
:10361000B8011F910F910C946F1A0F931F9341E003
:1036200050E060E070E004C0440F551F661F771F34
:103630008A95D2F740955095609570958091470294
:1036400090914802A0914902B0914A028A019B01DF
:10365000082319232A233B23C901B8011F910F9185
:103660000C946F1A0F931F9341E050E060E070E0FC
:1036700004C0440F551F661F771F8A95D2F78091AB
:10368000470290914802A0914902B0914A028A01F2
:103690009B01082719272A273B27C901B8011F9139
:1036A0000F910C946F1A0F931F9300914702109182
:1036B00048022091490230914A02602B712B822BE3
:1036C000932B1F910F910C946F1A0F931F930091DE
:1036D0004702109148022091490230914A0260232A
:1036E0007123822393231F910F910C946F1A0F93D0
:1036F0001F93009147021091480220914902309196
:103700004A0260277127822793271F910F910C94FB
:103710006F1A08958F929F92AF92BF92DF92EF92AD
:10372000FF920F931F93CF93DF9300D000D01F928F
:10373000CDB7DEB76B837C838D838A018C819D81BD
:10374000892B21F01F3F29F44F3F19F480E090E0CE
:103750004CC08B818823C9F180904B0290904C0221
:10376000A0904D02B0904E02809147029091480285
:10377000A0914902B0914A02882A992AAA2ABB2A12
:103780008FE1E82EF12CD501C4010E2C04C0B695B2
:10379000A795979587950A94D2F780FF07C0DE2CEE
:1037A000B8018E2D0E94DE1D019729F481E0E81AF0
:1037B000F10848F7D12C88E0189FF0011124E00FA0
:1037C000F11DE953FE4FD08209C088E0189FF00137
:1037D0001124E00FF11DE953FE4FD08009831A83B5
:1037E00069817A818D2D0E94DE1D0F900F900F90C0
:1037F0000F900F90DF91CF911F910F91FF90EF905D
:10380000DF90BF90AF909F908F90089520910B0113
:1038100030910C01F90132969FEF40E05191581719
:1038200089F09F3F19F4511101C0942F4F5F46302A
:10383000A9F79F3F39F0F901E90FF11D97FDFA95BE
:1038400082830895089520910B0130910C01F901B4
:103850003296285F3F4F9081981301C010823196B5
:10386000E217F307C1F7089581E090E0E0910B01C2
:10387000F0910C01E80FF91F108201968830910534
:10388000A9F7089580915902089590915902892BC2
:1038900080935902089580959091590289238093CD
:1038A000590208958093590208951092590208957B
:1038B00090915802892B8093580208958095909199
:1038C000580289238093580208951092580208954F
:1038D00080934F02089510924F02089580910B013A
:1038E00090910C01FC0131969C01285F3F4F80E0D4
:1038F000919191118F5FE217F307D1F70895E0914D
:103900000B01F0910C01809159028083E0910B0131
:10391000F0910C01908180915802892B80838091D5
:103920004F02882361F0E0910B01F0910C0190812E
:10393000892B80830E946E1C811110924F0280910E
:103940000B0190910C010C94931090933301809390
:10395000320108958295982F9C7C392F36953695A3
:10396000282F237344E0249FC0011124932F982B08
:10397000292F2A7A2695892F8575880F822B0895FD
:103980000895CF93DF9300D000D01F92CDB7DEB75C
:103990000F900F900F900F900F90DF91CF9108959F
:1039A000089508950C94EC1180916F02843021F1F8
:1039B00010925B0220E488E190E00FB6F894A8959D
:1039C000809360000FBE2093600083B7817F846086
:1039D00083BF83B7816083BF7894889583B78E7FD8
:1039E00083BF0FB6F894A89580916000886180939A
:1039F0006000109260000FBE0895CF930E942212C3
:103A00000E94A0060E942312C0E08C2F0E9419067B
:103A1000811104C0CF5FC031C1F701C081E0CF91F7
:103A200008950E941F060C9451161F920F920FB614
:103A30000F9211248F939F93AF93BF9380915B025A
:103A4000811113C080915C0290915D02A0915E0291
:103A5000B0915F024196A11DB11D80935C029093CD
:103A60005D02A0935E02B0935F02BF91AF919F9100
:103A70008F910F900FBE0F901F90189582E084BD1C
:103A800093E095BD9AEF97BD80936E0008952FB790
:103A9000F89480915C0290915D02A0915E02B091D9
:103AA0005F022FBF08952FB7F89460915C02709168
:103AB0005D0280915E0290915F022FBF0895CF92C8
:103AC000DF92EF92FF920F931F932FB7F8944091DC
:103AD0005C0250915D0260915E0270915F022FBFA7
:103AE0006A017B01EE24FF248C0120E030E0C01647
:103AF000D106E206F30610F4415051099A01281B41
:103B0000390BC9011F910F91FF90EF90DF90CF907B
:103B100008951F920F920FB60F9211248F939F93C7
:103B2000AF93BF9380915C0290915D02A0915E0281
:103B3000B0915F020196A11DB11D80935C0290932C
:103B40005D02A0935E02B0935F02BF91AF919F911F
:103B50008F910F900FBE0F901F9018950E94A00D8F
:103B6000F8942FEF87EA91E6215080409040E1F7EA
:103B700000C0000087E090EBDC0180937802909316
:103B80007902A0937A02B0937B029CE088E10FB6A1
:103B9000F894A895809360000FBE90936000FFCFCB
:103BA00028E0929FF0011124E80FF11DE052FF4F31
:103BB0009491892F8F7092959F700895CF93C82FFD
:103BC000CB010E94D01D282F30E080E1989FA001FA
:103BD0001124422B532B4038510519F480E090E01A
:103BE00015C09770E92FF0E088E0C89FE00DF11D47
:103BF000112484E0EE0FFF1F8A95E1F7E20FF31F17
:103C0000EE0FFF1FE050F84985919491CF910895F0
:103C100080E090E0089508958091620280FF0BC0DB
:103C20006091100185E0689FB0011124759567953A
:103C3000759567952BC081FF09C06091100185E0E3
:103C4000689FB00111247595679520C082FF07C059
:103C50006091100185E0689FB001112417C0909118
:103C600063029923D1F060910F01961788F7209194
:103C7000100185E0289F90011124929FA001939F3D
:103C8000500D112470E0CA010E94C82560387105EA
:103C900040F46115710539F002C065E070E0862FCF
:103CA00008958FE7089581E008958091620280FF72
:103CB00008C060910E0170E07595679575956795E0
:103CC00021C081FF06C060910E0170E07595679577
:103CD00019C082FF04C060910E0170E010C0909185
:103CE00063029923C1F060910D019617A0F78091AE
:103CF0000E01899FC001112470E00E94C825603820
:103D0000710528F46115710521F0862F08958FE75C
:103D1000089581E0089561E070E0F4CF803F21F4E0
:103D20000E940C1E819504C0813F29F40E940C1E44
:103D3000809366020895823F21F40E940C1E8195B3
:103D400004C0833F29F40E940C1E809365020895ED
:103D5000893F19F40E94551E05C08A3F31F40E9424
:103D6000551E81958093670208958B3F21F40E9430
:103D7000551E819504C08C3F29F40E94551E8093E6
:103D800068020895843F21F480916402816017C025
:103D9000853F21F480916402826011C0863F21F446
:103DA0008091640284600BC0873F21F4809164029B
:103DB000886005C0883F31F48091640280618093FF
:103DC000640208958D3F21F48091620281600BC0EE
:103DD0008E3F21F480916202826005C08F3F29F4FA
:103DE000809162028460809362020895803F39F47A
:103DF0008091660287FF6CC01092660269C0813FA5
:103E000029F4809166021816BCF362C09091650295
:103E1000823F29F497FF5CC01092650259C0833F2E
:103E200019F41916CCF354C0893F41F4809167020C
:103E300018160CF04DC0109267024AC08A3F29F450
:103E40008091670287FF44C0F6CF8B3F39F48091A1
:103E5000680287FF3DC0109268023AC08C3F29F487
:103E6000809168021816BCF333C0843F21F480911E
:103E700064028E7F17C0853F21F4809164028D7F9C
:103E800011C0863F21F4809164028B7F0BC0873F75
:103E900021F480916402877F05C0883F31F48091CE
:103EA00064028F7E8093640213C08D3F21F4809161
:103EB00062028E7F0BC08E3F21F4809162028D7F63
:103EC00005C08F3F29F4809162028B7F809362024C
:103ED0008091650281110EC08091660281110AC035
:103EE00080916702811106C080916802811102C031
:103EF00010926302089580915A0283FF7EC08BE482
:103F000094E00E947505809164021F928F9386E46D
:103F100094E09F938F930E940E0684E494E00E94A5
:103F2000750580916502282F082E000C330B3F93F6
:103F30008F9381E494E09F938F930E940E068FE30A
:103F400094E00E94750580916602282F082E000CCF
:103F5000330B3F938F938CE394E09F938F930E9456
:103F60000E068AE394E00E94750580916702282F6F
:103F7000082E000C330B3F938F9387E394E09F93BD
:103F80008F930E940E0685E394E00E947505809150
:103F90006802282F082E000C330B3F938F9382E387
:103FA00094E09F938F930E940E068FE294E00E940C
:103FB0007505809163021F928F938CE294E09F932A
:103FC0008F930E940E068AE294E00E94750580910C
:103FD00062021F928F9387E294E09F938F930E94D7
:103FE0000E0684E294E00E9475058DB79EB74C964C
:103FF0000FB6F8949EBF0FBE8DBF84E692E00E947C
:10400000DC100E94471D9093610280936002089526
:104010001F93CF93DF9380916002909161020E9481
:104020005F1DAC0190916302992321F02091110151
:1040300030E006C0209112018AE0289F90011124EF
:104040004217530708F485C080916502C09166024B
:10405000D091670210916802811107C0C11175C02B
:10406000D11173C0111171C074C09F3F19F09F5FCF
:1040700090936302181624F40E940C1E809365022C
:104080008091650287FF05C00E940C1E8195809378
:1040900065021C1624F40E940C1E80936602809117
:1040A000660287FF05C00E940C1E81958093660200
:1040B00060916502662331F1C0916602CC2311F153
:1040C000062E000C770B880B990B0E94C32423E368
:1040D00033E343E35FE30E9427250E948B24609330
:1040E00065026C2FCC0F770B880B990B0E94C324B1
:1040F00023E333E343E35FE30E9427250E948B24FD
:10410000609366021D1624F40E94551E8093670278
:104110008091670287FF05C00E94551E819580939C
:104120006702111624F40E94551E80936802809144
:10413000680287FF05C00E94551E81958093680222
:10414000DF91CF911F910C947B1F9F3F09F08FCF80
:1041500097CFDF91CF911F910895E4E6F2E085E0DB
:10416000DF011D928A95E9F71092630210926202B4
:1041700008958EE696E00E9475051F9281E08F9368
:104180001F9285E08F9380E296E09F938F930E9429
:104190000E060F900F900F900F900F900F900895B4
:1041A0008330E9F128F4813061F0823009F108951B
:1041B000853009F462C008F449C0863009F474C03F
:1041C000089580911201262F30E0280F311D2F3FD6
:1041D000310524F4680F6093120103C08FEF8093C0
:1041E0001201809112011F928F9389E595E072C0B0
:1041F00080911101262F30E0280F311D2F3F31050E
:1042000024F4680F6093110103C08FEF80931101B4
:10421000809111011F928F9387E495E05BC080919C
:104220001001262F30E0280F311D2F3F310524F4D7
:10423000680F6093100103C08FEF8093100180918D
:1042400010011F928F9384E395E044C080910F0189
:10425000262F30E0280F311D2F3F310524F4680F41
:1042600060930F0103C08FEF80930F0180910F01C6
:104270001F928F938FE195E02DC080910E01262F24
:1042800030E0280F311D2F3F310524F4680F609373
:104290000E0103C08FEF80930E0180910E011F92DB
:1042A0008F9386E095E016C080910D01262F30E0B7
:1042B000280F311D2F3F310524F4680F60930D0145
:1042C00003C08FEF80930D0180910D011F928F939A
:1042D0008BEE94E09F938F930E940E060F900F90A9
:1042E0000F900F900895833081F128F4813059F0B8
:1042F0008230D1F00895853009F449C0B8F1863094
:1043000009F456C0089580911201681720F4861BA5
:104310008093120102C010921201809112011F922B
:104320008F938CED94E054C080911101681720F4B4
:10433000861B8093110102C010921101809111011E
:104340001F928F938AEC94E043C08091100168170C
:1043500020F4861B8093100102C0109210018091FE
:1043600010011F928F9387EB94E032C080910F0170
:10437000681720F4861B80930F0102C010920F0172
:1043800080910F011F928F9382EA94E021C0809167
:104390000E01681720F4861B80930E0102C0109254
:1043A0000E0180910E011F928F9389E894E010C056
:1043B00080910D01681720F4861B80930D0102C0C7
:1043C00010920D0180910D011F928F938EE694E063
:1043D0009F938F930E940E060F900F900F900F9057
:1043E0000895CF93C82F1F928F9383E797E09F93F1
:1043F0008F930E940E0681E090E0A0E0B0E0BC0147
:10440000CD0104C0660F771F881F991FCA95D2F788
:104410000E947A1A0F900F900F900F90CF910C94EA
:104420005116CF93873288F58E3108F00BC18E304C
:1044300009F487C0D8F4873009F460C08B3009F4E0
:104440004FC0863009F002C180915A02817F8E7F71
:1044500080935A0288E797E00E9475058BE39AE003
:104460000E94750581E080936A0246C0863109F496
:10447000B0C020F4803109F47AC0E8C0893109F471
:1044800091C08B3109F449C0E1C0883349F150F43F
:10449000893209F4D5C0853309F4D2C0873209F0D6
:1044A000D5C0CEC0833409F4CBC028F48A3308F4D5
:1044B000CDC08953C8C0883409F0C8C00E945116C5
:1044C0008AE29AE00E9475052FEF83ED90E3215078
:1044D00080409040E1F700C000000E94AE1D0CC07B
:1044E0008FE997E041C081E19AE00E9475058091D3
:1044F0005A02816080935A02C1E0ADC080915A0295
:10450000C82FC17080FFEFCF8DE19AE00E94750542
:1045100080915A02817F8E7F3FC090915A0291FB19
:10452000CC27C0F981E0C827892FC0FB81F980938F
:104530005A02CC2319F084E09AE029C086EF99E072
:1045400013C090915A0292FBCC27C0F981E0C82792
:10455000892FC0FB82F980935A02CC2319F087EE91
:1045600099E015C087ED99E00E947505C5CF90913F
:104570005A0293FBCC27C0F981E0C827892FC0FBE2
:1045800083F980935A02CC2351F08BEC99E00E947E
:10459000750580915A02816080935A025CC08EEB4F
:1045A00099E0E2CF8FEA99E00E94750587E899E0EB
:1045B0000E9475058DE399E00E94750580E199E000
:1045C0000E9475058BEC98E00E9475058DE998E0D6
:1045D000CBCF8FE898E00E9475050E9487101F924C
:1045E0008F9385E798E09F938F930E940E068091AA
:1045F0000A011F928F938EE598E09F938F930E94FC
:104600000E06809177011F928F938BE498E09F9321
:104610008F930E940E060E94531D9F938F937F934A
:104620006F9384E398E09F938F930E940E068DB75B
:104630009EB742960FB6F8949EBF0FBE8DBF5CCF5B
:1046400080E001C08D510E94F12156CF82E398E0B5
:104650000E947505C0E08C2FCF91089580E00895E9
:1046600080E00895CF93C82F80916A02813081F055
:1046700020F0823009F44FC046C1E0910B01F09167
:104680000C018081813169F0823209F03EC109C09C
:10469000E0910B01F0910C018081813111F08232A7
:1046A00061F48C2F0E942E23811104C08C2F0E9454
:1046B00011222FC081E090E02CC08C2F0E9430236B
:1046C000811126C0C431E1F070F4CB3081F0C031EB
:1046D000D1F40E94B9208BE697E00E94750582E034
:1046E00080936A0215C0C93259F0C83361F488E773
:1046F00097E00E9475058FE697E00E94750508C057
:1047000010926A0204C189E697E00E947505FFC015
:1047100081E08170FEC0C43228F5CE3108F0C1C0FE
:10472000CB30A1F1D0F4C73009F0D3C08EE1809333
:10473000120182E3809311018AE08093100184E1E9
:1047400080930F0188E080930E0188E280930D0131
:104750008FE096E00E947505BFC0C33149F1C431B6
:10476000C1F0B7C0CB3409F4A9C028F4C93289F02C
:10477000C83361F0AEC0C13509F49EC0C23509F43A
:1047800099C0CE3409F0A5C06AE09EC00E94B9204D
:10479000A3C080916902882319F0109269029CC01D
:1047A0008CE196E00E94750581E080936A02B1C0B9
:1047B00086EF95E00E94750584EE95E00E947505F0
:1047C000809112011F928F9381EE95E09F938F93BA
:1047D0000E940E068FED95E00E9475058DEC95E028
:1047E0000E947505809111011F928F938AEC95E0CC
:1047F0009F938F930E940E0688EC95E00E947505AA
:1048000089EB95E00E947505809110011F928F93AE
:1048100086EB95E09F938F930E940E0684EB95E0C4
:104820000E94750583EA95E00E94750580910F014D
:104830001F928F9380EA95E09F938F930E940E06BC
:104840008EE995E00E94750589E895E00E9475055E
:1048500080910E011F928F9386E895E09F938F932E
:104860000E940E0684E895E00E9475058DE695E0AD
:104870000E94750580910D011F928F938AE695E045
:104880009F938F930E940E0688E695E00E9475051F
:104890008DB79EB748960FB6F8949EBF0FBE8DBFDA
:1048A0001BC0CE51EC2FF0E0E85DFE4F808180937D
:1048B000690212C061E003C061E006C06AE0809155
:1048C00069020E94D02008C0809169020E94732171
:1048D00003C08DE096E013C080916902882369F0DF
:1048E0001F928F9387E096E09F938F930E940E060E
:1048F0000F900F900F900F9004C084E096E00E94FC
:10490000750581E006C010926A0280E002C080E076
:1049100000CFCF9108950E9492246894B1110C9415
:10492000212508950E94062588F09F5798F0B92FF9
:104930009927B751B0F0E1F0660F771F881F991FD4
:104940001AF0BA95C9F714C0B13091F00E94202531
:10495000B1E008950C942025672F782F8827B85F41
:1049600039F0B93FCCF3869577956795B395D9F72C
:104970003EF490958095709561957F4F8F4F9F4F36
:104980000895E89409C097FB3EF490958095709542
:1049900061957F4F8F4F9F4F9923A9F0F92F96E98B
:1049A000BB279395F695879577956795B795F11100
:1049B000F8CFFAF4BB0F11F460FF1BC06F5F7F4F9D
:1049C0008F4F9F4F16C0882311F096E911C07723AF
:1049D00021F09EE8872F762F05C0662371F096E8B8
:1049E000862F70E060E02AF09A95660F771F881F87
:1049F000DAF7880F9695879597F9089557FD90589F
:104A0000440F551F59F05F3F71F04795880F97FB92
:104A1000991F61F09F3F79F087950895121613064C
:104A20001406551FF2CF4695F1DF08C0161617067B
:104A30001806991FF1CF86957105610508940895B0
:104A4000E894BB2766277727CB0197F908950E9442
:104A50003A250C94AB250E949D2538F00E94A42590
:104A600020F0952311F00C9494250C949A25112490
:104A70000C9421250E94FE2470F3959FC1F3950F9D
:104A800050E0551F629FF001729FBB27F00DB11DD2
:104A9000639FAA27F00DB11DAA1F649F6627B00D62
:104AA000A11D661F829F2227B00DA11D621F739F4B
:104AB000B00DA11D621F839FA00D611D221F749F59
:104AC0003327A00D611D231F849F600D211D822FA0
:104AD000762F6A2F11249F5750409AF0F1F08823C7
:104AE0004AF0EE0FFF1FBB1F661F771F881F9150F4
:104AF0005040A9F79E3F510580F00C9494250C94EA
:104B000021255F3FE4F3983ED4F38695779567952A
:104B1000B795F795E7959F5FC1F7FE2B880F911D1D
:104B20009695879597F9089597F99F6780E870E0C3
:104B300060E008959FEF80EC089500240A94161613
:104B4000170618060906089500240A94121613067B
:104B5000140605060895092E0394000C11F4882309
:104B600052F0BB0F40F4BF2B11F460FF04C06F5F25
:104B70007F4F8F4F9F4F0895991B79E004C0991F75
:104B8000961708F0961B881F7A95C9F780950895A7
:104B900097FB072E16F4009407D077FD09D00E94EA
:104BA000E22507FC05D03EF4909581959F4F08952E
:104BB000709561957F4F0895EE0FFF1F0590F4915A
:104BC000E02D0994AA1BBB1B51E107C0AA1FBB1F04
:104BD000A617B70710F0A61BB70B881F991F5A9589
:104BE000A9F780959095BC01CD010895F894FFCF69
:104BF000E108D209AF097B094709015002280814CE
:104C00000A321E404D36228C033F030903E702732C
:104C1000028C02A502BE0200010203040506070879
:024C2000090089
:106800008800EA44E944E244040005000600070069
:10681000080009000A000B000C000D000E000F001C
:1068200010001100120013001400150016001700CC
:10683000180019001A001B001C001D001E001F007C
:10684000200021002200230024002500260027002C
:10685000280029002A002B002C002D002E002F00DC
:10686000300031003200330034003500360037008C
:10687000380039003A003B003C003D003E003F003C
:1068800040004100420043004400450046004700EC
:10689000480049004A004B004C004D004E004F009C
:1068A000500051005200530054005500560057004C
:1068B000580059005A005B005C005D005E005F00FC
:1068C000600061006200630064006500850067008D
:1068D000680069006A006B006C006D006E006F005C
:1068E0007000710072007300890087008A008B00BD
:1068F000E000E100E200E300F1A1E500E600E700CE
:106900000100010001000100EA4401000100E2442D
:106910000100010001000100460001004A004B0097
:10692000010001004700480001000100E9440100A6
:106930000100010001000100010001003A003B00DC
:106940003C003D003E003F0040004100420043004B
:10695000010035004C0039000100440045005200A0
:1069600049000100010050004F0029004D004E0079
:1069700051000100680069006A006B006C006D0046
:106980006E006F0070007100720073000100010062
:1069900001000100010001000100010001004D00A3
:1069A0004A004E004B0001000100010001000100FF
:1069B00001000100010001000100010001000100CF
:1069C00001000100010001000100010001000100BF
:1069D00001000100010001000100010001000100AF
:1069E0000100010001000100490001000100010057
:1069F000010001000100010001000100010001008F
:00000001FF
